:100000000C94B9030C94F1030C94F1030C94F103D8
:100010000C94F1030C94F1030C94F1030C94F10390
:100020000C94F1030C94F1030C94F1030C946027ED
:100030000C940F280C9430220C94F1030C94F103CF
:100040000C94F1030C94F1030C94F1030C94B92279
:100050000C94F1030C94F1030C94F1030C94F10350
:100060000C94F1030C94F1030C94F1030C94F10340
:100070000C94F1038A068A06B606B60624071E0803
:100080001E081E084207AA07BB07BB077A1A7D1A7B
:10009000821A891A8E1A931A981A9D1AA21AA71AE6
:1000A000AC1AB11AB31AB61AB91ABC1ABF1AC21AC4
:1000B000C41AC71ACB1A541C571C811C941C9C1CB4
:1000C000A71CAA1CAA1CAA1CF21CF21CAF1CB21C66
:1000D000B71CC41CD11CD41CD81CE51C531DC51D49
:1000E0005B1D251D291D5F1D2C1D621D6D1D371DEE
:1000F000BB1D3B1D711D3F1D751D9F1D431D791DA2
:10010000A91D491D7F1D891D301D661D331D691DDB
:100110004E1D841D951DB51DB71D211D571DCE1DDE
:1001200004210A21F820FE20102116211C21772805
:100130009E2896299E289629EA280D299629642921
:10014000732929001E001F00200021002200230027
:1001500024002500260027002D002E0000002B0083
:1001600014001A000800150017001C0018000C00ED
:10017000120013002F0030003100E00004001600D0
:10018000070009000A000B000D000E000F003300ED
:10019000340000002800E10000001D001B000600E4
:1001A000190005001100100036003700380000006B
:1001B000E500E000E3000000E20000002C00000089
:1001C000E600E70000006500215200002A00007CE4
:1001D0003A003B003C003D003E003F004000410033
:1001E0004200430044004500010001002A00520083
:1001F00028000100010001000100460047004800FE
:100200005200010001003900500051004F00A800C9
:100210000100550054004A004B0050004F000100FF
:10022000010001000100AC00AE00AB00AA00A90073
:10023000570056004D004E00510001000100010022
:10024000010001000100010001000100BE00BD002D
:1002500001000100010001004C000100010001004B
:100260000100010001000100010001000100010086
:100270000100010001000100010001000100010076
:100280000100010001000100010001000100010066
:100290000100010001000100010001000100010056
:1002A0000100010001000100010001000100010046
:1002B0000100010001000100010001000100010036
:1002C0000100010001000100010001000100010026
:1002D0000100010001000100010001000100010016
:1002E0000100010001000100010001000100010006
:1002F00001000100010001000100010001000100F6
:1003000001000100010001000100010001000100E5
:1003100001000100010001000100010001000100D5
:1003200001000100010001000100010001000100C5
:1003300001000100010001000100010001000100B5
:1003400001000100010001000100010001000100A5
:100350000100010001000100010001000100010095
:100360000100010001000100010001000100010085
:1003700001001E0F0500047F3F1F64321464321415
:10038000783C1E1E140A052223252628292A2C2DF6
:100390002F3032333536383A3B3D3E4042434547B5
:1003A000494A4C4E5051535557595A5C5E606264ED
:1003B0006668696B6D6F71737577797B7D7F8183FB
:1003C0008587898A8C8E90929496989A9C9E9FA1FC
:1003D000A3A5A7A8AAACAEAFB1B3B4B6B8B9BBBC1D
:1003E000BEBFC1C2C3C5C6C7C9CACBCCCDCED0D192
:1003F000D2D2D3D4D5D6D7D7D8D9D9DADADBDBDB8A
:10040000DCDCDCDCDCDDDDDDDDDCDCDCDCDCDBDB2A
:10041000DBDADAD9D9D8D7D7D6D5D4D3D2D2D1D07E
:10042000CECDCCCBCAC9C7C6C5C3C2C1BFBEBCBB7B
:10043000B9B8B6B4B3B1AFAEACAAA8A7A5A3A19FF3
:100440009E9C9A98969492908E8C8A8987858381B7
:100450007F7D7B79777573716F6D6B696866646298
:10046000605E5C5A5957555351504E4C4A49474566
:100470004342403E3D3B3A3836353332302F2D2C07
:100480002A292826252322FFAA7F554000010101A1
:100490000101010101010202020202020202020341
:1004A0000303030303030304040404040404050511
:1004B00005050506060606060707070707080808D4
:1004C00008090909090A0A0A0B0B0B0C0C0C0D0D83
:1004D0000D0E0E0E0F0F0F1010111111121213131B
:1004E0001414151516161717181819191A1A1B1B94
:1004F0001C1D1D1E1E1F20202122222324242526F0
:1005000026272829292A2B2C2D2D2E2F3031323227
:10051000333435363738393A3B3C3D3E3F40414233
:10052000434445464748494A4C4D4E4F5051535419
:10053000555658595A5B5D5E5F61626465666869CD
:100540006B6C6D6F7072737577787A7B7D7E80824D
:10055000838587888A8C8E8F91939596989A9C9E96
:10056000A0A2A3A5A7A9ABADAFB1B3B5B7BABCBEA6
:10057000C0C2C4C6C9CBCDCFD1D4D6D8DBDDDFE273
:10058000E4E7E9EBEEF0F3F5F8FAFDFF0000000018
:10059000000000002A2B28000000000000000000DE
:1005A0000000000000000029000000002C1E342084
:1005B000212224342627252E362D3738271E1F20AA
:1005C0002122232425263333362E37381F040506EF
:1005D0000708090A0B0C0D0E0F1011121314151633
:1005E0001718191A1B1C1D2F3130232D3504050631
:1005F0000708090A0B0C0D0E0F1011121314151613
:100600001718191A1B1C1D2F3130354C0000000023
:1006100000000000000000000000000000000000DA
:1006200000000000000000000000000000000000CA
:100630007E0F00D4FFFFFFC7000000781E035300A9
:100640007400650065007A007900360030002000F3
:100650005200650076002000410000000E033400C7
:10066000700070006C006500740000000403090451
:1006700009025B00030100A0FA0904000001030164
:100680000100092111010001224000070581030832
:10069000000109040100020300000009211101000A
:1006A0000122220007058203200001070503032021
:1006B00000010904020001030000000921110100EA
:1006C000012232000705840320000112010002000C
:1006D000000008444402000100010200010660FF1E
:1006E0000961A1010962150026FF009520750881A6
:1006F000020963150026FF00952075089102C005C8
:10070000010980A101850319012AB700150126B747
:1007100000950175108100C0050C0901A101850437
:1007200019012AA002150126A00295017510810069
:10073000C005010906A101050719E029E7150025F3
:100740000195087501810295017508810105071958
:100750000029FF150026FF00950675088100050891
:1007600019012905950575019102950175039101FE
:10077000C00011241FBECFEFD4E0DEBFCDBF04B652
:1007800003FE18C08091110390911203A0911303EE
:10079000B09114038730904BA740B04B59F410929E
:1007A0001103109212031092130310921403E0E04D
:1007B000F8E3099511E0A0E0B1E0E2E1F7E502C05D
:1007C00005900D92AA3DB107D9F723E0AAEDB1E05B
:1007D00001C01D92A131B207E1F70E941E130C94D3
:1007E000872B0C94000084E00895282F8430E8F4CF
:1007F0006530D8F44E30C8F4862F90E06EE070E09B
:100800000E94CD29FC01822F90E066E470E00E94F6
:10081000CD298E0F9F1FFC01E40FF11DEE0FFF1F6E
:10082000EE5BFE4F85919491089580E090E00895ED
:1008300081E0089581E008950E941A0408950895C2
:100840000E941F040895A5E0B0E0E9E2F4E00C94F2
:10085000772A49835A833091E10189819A81311144
:1008600014C0662359F0222349F00E94D809182F9A
:10087000682F89819A810E94AF0903C00E94C40930
:10088000182F69817A81812F04C00E94D80969815B
:100890007A810E949E102596E3E00C94932AFC0135
:1008A000262F408151816281738184810E942304BB
:1008B000089581E00895CF93DF93EC0160E00E94FA
:1008C0004F04BE010E942004DF91CF910895E1E022
:1008D000F0E0DF0102C0AA0FBB1F6A95E2F7BD017D
:1008E000DF0102C0AA0FBB1F4A95E2F7AD01462BFC
:1008F00001C0EE0F2A95EAF7942F9823491302C0FE
:100900008E2B0895E0958E230895242F462F682F6F
:100910008091FD010E9467040E94110908950E94C0
:10092000E21108950E94DC11089508950E949D0827
:100930000E9495042FEF84E39CE02150804090407A
:10094000E1F700C0000008950E9496040E94DF2293
:1009500008950E9496040E94032308950F931F9305
:10096000CF93DF938C0161E00E944F04EC01B8014A
:100970000E946F1B882309F450C0B801CE010E9469
:100980001C04882309F449C0B801CE010E94EC2060
:10099000882309F442C0B801CE010E94FD1C8823BF
:1009A000E1F1B801CE010E9452208823B1F1B801D3
:1009B000CE010E94641A882381F1F8018281882384
:1009C00041F1C3308CE7D807D1F040F4C115FCE702
:1009D000DF0791F0C130DC47A1F01BC0CB35ECE75D
:1009E000DE07A9F0CC35FCE7DF0771F0CA35DC473C
:1009F00081F40E94150E0DC00E94A4040EC00E9436
:100A00001D0E0E94A90409C00E940B0E02C00E9484
:100A1000190EC8010E94180401C080E0DF91CF9137
:100A20001F910F9108950E940E220E943D05089586
:100A30000E9441050E941722089508950E941D05F5
:100A4000089581E008950895CF93DF93D82F0E94F1
:100A50002105C82F882319F08D2F0E9423058C2F84
:100A6000DF91CF9108950895CF93C82F0E941E055E
:100A70008C2F0E942405CF91089580E00E943405B8
:100A800008950E9439210E9434050895CF930E9451
:100A90003921C82F8091DC01C81779F0C093DC019F
:100AA0000E949E226093DD017093DE018093DF013E
:100AB0009093E0018C2F0E943405CF910895ABE014
:100AC000B0E0E5E6F5E00C94782A4F835887698713
:100AD0007A878B8761110E94530D9E012F5F3F4FD4
:100AE00086E0F90111928A95E9F785E0FE013796D3
:100AF000D90101900D928A95E1F789819A814C8103
:100B00005D81452B31F09F3F31F491E08F3F19F427
:100B100003C091E001C090E090FF09C049815A8173
:100B20006B817C818D819E810E94780C05C0C901FA
:100B30000E9459048111F2CF2B96E2E00C94942A82
:100B4000FC01808191810E94050A0895CF9388233A
:100B500009F447C0C82F8CEF8C0F813AD0F46C2F6A
:100B600080910401909105010E94A721882349F0FA
:100B70006C2F80910401909105010E94E0210E9458
:100B8000770D6C2F80910401909105010E94DD2169
:100B90000CC080E28C0F883058F4C77081E001C02F
:100BA000880FCA95EAF70E94360D0E94770D19C08A
:100BB000EBE5EC0FE33040F4F0E0EC5AFE4F8081BF
:100BC00090E00E9451210DC0C85AC93150F4EC2F59
:100BD000F0E0EE0FFF1FEE5DFE4F808191810E94DD
:100BE0007621CF910895882359F1682F8CEF860FD5
:100BF000813A38F480910401909105010E94E0212E
:100C00000CC080E2860F883058F4677081E001C024
:100C1000880F6A95EAF70E943C0D0E94770D0895AF
:100C20008BE5860F833028F480E090E00E9451210C
:100C30000895685A693120F480E090E00E9476219E
:100C400008951F93CF93DF93182FEB010E94A60501
:100C5000209741F08FE99FE00197F1F700C0000075
:100C60002197F6CF812F0E94F305DF91CF911F913D
:100C70000895893319F060E070E002C060E570E02B
:100C80000E9421060895882321F00E94360D0E94BB
:100C9000770D0895882321F00E943C0D0E94770D66
:100CA0000895A0E0B0E0E7E5F6E00C94722A7C013C
:100CB000162FC72FFC01D281058102950F700E946B
:100CC0002C0D8823B9F0DD23A9F08C2F807F803490
:100CD00021F080E2810F883068F08091C20282FFAB
:100CE00009C082E00E94D90D0E942C0D91E0D82EFF
:100CF000D92601C0D12CCC2EC2948FE0C8228C2DD5
:100D000090E08C30910508F099C1FC01E65CFF4F42
:100D10000C945B2A8C2F807FCF70882311F0C295B2
:100D2000C07FDD2399F0CC2309F474C180E2810FE8
:100D3000883010F0111104C08C2F0E94360D03C0B2
:100D40008C2F0E94460D0E94770D64C1812F0E9456
:100D5000F305CC2309F472C180E2810F883038F1A9
:100D6000112329F18C2F0E944C0D24C08C2F807FE1
:100D7000CF70803211F0C295C07F112319F011306D
:100D8000D1F143C08091C20282FD17C0DD2349F03A
:100D9000CC2329F08C2F0E94360D0E94770D80E025
:100DA0003AC180E00E94F305CC2309F447C18C2F9F
:100DB0000E943C0D0E94770D41C1DD2371F000239C
:100DC00041F0013031F40E94560D8C2B0E94600DD1
:100DD00035C10E94560D8C2B23C0011103C00E9407
:100DE0006D0D2EC0013009F429C18C2F0E944A06D6
:100DF0000E946D0D23C1DD2321F0063008F01EC1D5
:100E00000EC0053008F01AC11BC0DD2361F00023BD
:100E100031F0F701858180FFFDC08F7085838C2FB5
:100E20000E9443060BC1002359F0193309F003C196
:100E3000FFEF27EE83E0F15020408040E1F7F9C05A
:100E40008C2F0E944A06FAC08C2F86958695837057
:100E500019F0813061F0F2C0DD2321F0812F9C2F49
:100E6000937002C080E090E00E945121EFC0DD232A
:100E700021F0812F9C2F937002C080E090E00E94AF
:100E80007621E4C08C2F837079F5D111DBC0412F1E
:100E9000429546954770440F440F212F2F70042E22
:100EA00001C0220F0A94EAF714FF08C08FE090E017
:100EB00001C0880F4A95EAF7809501C080E0C69589
:100EC000C695C370822BC23049F058F4C13019F076
:100ED0000E940209B7C00E94FC08B4C00E94080921
:100EE000B1C00E94F908AEC0DD2319F08C2F8170CB
:100EF00001C08695882309F4A5C0412F42954695E7
:100F00004770440F440F212F2F70042E01C0220F71
:100F10000A94EAF714FF08C08FE090E001C0880F40
:100F20004A95EAF7809501C080E0C695C695C370E2
:100F3000822BC23049F058F4C13019F00E944E099A
:100F400081C00E9448097EC00E9454097BC00E9453
:100F5000110978C0CF70DD2339F08C2F0E9423094E
:100F6000812F0E9443066EC0812F0E944A068C2F5B
:100F70000E942F0967C0123F21F128F4103F41F071
:100F8000113FC1F043C0133F19F1143F79F03EC047
:100F9000DD2341F0053008F051C08C2F8F710E9485
:100FA0003C094CC0063008F049C0F7CF8091C2021E
:100FB00082FD18C0DD2339F08C2F8F710E94230928
:100FC0003DC0DD23C9F38C2F8F710E942F0936C0DD
:100FD000DD2329F08C2F8F710E941A092FC00E94E7
:100FE00016092CC0DD2349F0CF718C2F0E942309F4
:100FF00063E08C2F0E94BB0D21C081E00E94D90DBF
:101000000230E0F082E00E94D90D18C0DD2331F0FB
:10101000002391F2812F0E94A60510C0002399F2AF
:10102000193349F49FEFE7EEF3E09150E040F040D0
:10103000E1F700C00000812F0E94F30588EF8C0DBE
:10104000843020F40E9439210E943405DD2089F08B
:101050000E94280D80FD0DC0F70112820E94220D12
:101060000E942309C7010E9456080E94220D0E9477
:101070002F09CDB7DEB7E8E00C948E2A0F931F93AB
:10108000CF93DF93EC01688179818A810E94100AF5
:101090008C010E945A090E94EC08B801CE010E94FE
:1010A0005106DF91CF911F910F910895CF93DF9358
:1010B000EC01988189812B813C81232B31F08F3F7A
:1010C00031F481E09F3F19F403C081E001C080E06A
:1010D00080FD1AC0CE010E94AE0481110FC00E9493
:1010E0002C0D882389F08A81882371F08091C202B7
:1010F00082FF0AC082E00E94D90D06C0CE010E9484
:101100003E08CE010E945B04DF91CF91089580E0FC
:1011100090E00E94512180E090E00E9476210E94A0
:10112000530D0E94770D089580910401909105015F
:101130000E94E3210E94870808950E94430D0E94A7
:101140009408089592959F70963079F010F492501B
:1011500001C09A50923068F4803F69F018F4883EDC
:1011600040F409C0843F29F406C0883E20F0813F46
:1011700011F080E0089581E00895FC019081818163
:1011800023813481232B31F08F3F31F481E09F3F65
:1011900019F403C081E001C080E080FD07C08081B8
:1011A00091810E94050A0E94A208089580E0089596
:1011B000A5E0B0E0EEEDF8E00C94782A2596E2E0A8
:1011C0000C94942AA6E0B0E0E8EEF8E00C94782ABB
:1011D0002696E2E00C94942A089508950E94ED0862
:1011E00008950E94EE0808950E94F1088093FE0180
:1011F00008950E94F40808959091FE01892B0E94A1
:10120000F40808959091FE0189230E94F40808953E
:101210009091FE0189270E94F40808950E94ED082C
:1012200008950E940E098093FD01089580E00E94B8
:101230001109089591E001C0990F8A95EAF7892F65
:101240000E941109089521E030E001C0220F8A9523
:10125000EAF78091FD01822B0E941109089521E097
:1012600030E001C0220F8A95EAF720958091FD01B8
:1012700082230E941109089521E030E001C0220F6D
:101280008A95EAF78091FD0182270E94110908954D
:101290009091FD01892B0E94110908959091FD0103
:1012A00089230E94110908959091FD0189270E94C8
:1012B000110908950895282FFA01862F8770A1E05B
:1012C00001C0AA0F8A95EAF7CB0133E0969587957E
:1012D0003A95E1F763E070E00E94CD29E80FF91F2D
:1012E00040E050E0622F70E090819B01042E02C02C
:1012F000369527950A94E2F72170219529272A230C
:10130000292721934F5F5F4F4330510569F70895B7
:10131000FB01A82FA77023E0969587952A95E1F702
:1013200063E070E00E94CD29E80FF91F40E050E033
:1013300080E0219130E00A2E02C0369527950A946C
:10134000E2F721703327042E01C0220F0A94EAF736
:10135000822B4F5F5F4F4330510559F70895953009
:1013600090F48E3080F4362F282F892F90E06EE095
:1013700070E00E94CD29BC01620F711D42EE51E068
:10138000832F0E945B090895953080F48E3070F4AD
:10139000282F892F90E06EE070E00E94CD2962EE48
:1013A00071E0820F911D0E948809089580E00895E0
:1013B000CF92DF92FF920F931F93CF93DF936C0135
:1013C0000091FD018091FE01082BC7E0D0E010E004
:1013D000C8010C2E02C0959587950A94E2F780FD0E
:1013E00004C02197A8F7F12C07C0FC2EB6018C2F62
:1013F0000E94AA100197A9F38F2DDF91CF911F9121
:101400000F91FF90DF90CF900895CF93DF93EC0181
:101410000E94D809BE010E94AA10DF91CF910895C1
:101420001F93CF93DF93EB019091E101992321F07A
:10143000CB010E94050A13C0882349F0CB010E940A
:10144000D809182F682FCE010E94AF0904C0CB0124
:101450000E94C409182FBE01812F0E94AA10DF919B
:10146000CF911F910895CF93DF93C091FF01809199
:101470000002C817A1F0D0E0CE0166E070E00E9443
:10148000CD29FC01EF5FFD4F408151816281738165
:10149000848195810E94E2082196C770E8CFDF9190
:1014A000CF91089540913102509132026091330200
:1014B0007091340280913502909136020E94E208C8
:1014C00008951F93CF93DF938091360282958F709A
:1014D00009F05AC080913302882309F455C0209145
:1014E000FF0110910002C0913102D0913202A0910F
:1014F0003402B091350281E0CF3F09F080E0482FFF
:10150000211709F441C0109721F0DF3F21F080E05E
:1015100003C081E001C0842F30E080FD31C0C901EB
:1015200066E070E00E94CD29FC01EF5FFD4F8181F4
:101530008D1326C080818C1323C08281811120C02D
:10154000838194818A1B9B0B883C9105C8F4809110
:1015500036028F70806180933602C90166E070E0C8
:101560000E94CD29FC01EA5FFD4F90819F70906140
:10157000908381E392E00E9456080E94330A04C0DF
:101580002F5F3F4F2770BCCFDF91CF911F91089500
:10159000A1E1B0E0EEECFAE00C946F2A8C0185E05A
:1015A000F801DE011D9601900D928A95E1F7F80190
:1015B000E280909131023091320260913402709158
:1015C00035026115710531F03F3F31F481E09F3FF5
:1015D00019F403C081E001C080E0F82FF1709F2E64
:1015E00080FD44C1F80140812181A380B48081E362
:1015F000C82E82E0D82EF0903302F501E61BF70BDF
:10160000FF2009F4DDC080913602582F507FE83C5E
:10161000F10508F097C0511156C0231313C04913A8
:1016200011C0FE2CE1100EC08F70806180933602D5
:101630000E94520AC6010E94560880913602F801A3
:10164000858351C1A114B10431F02F3F31F481E001
:101650004F3F19F403C081E001C080E080FD03C06A
:1016600081E08E2502C080E090E0F82FF170FF2E1F
:1016700080FF1FC0E091FF0130910002E31709F4E1
:1016800010C1F0E0CF0166E070E00E94CD29DC01DE
:10169000AF5FBD4F11968C911197281307C08C91A5
:1016A000481304C012968C91E81203C03196E7707B
:1016B000E5CFFE2CEE2009F416C180913602816040
:1016C0008093360254C0231306C0491304C0E110AE
:1016D00002C0F80199C0C8010E94BD08882361F1C9
:1016E000EE2051F120913602822F82958F7090E08A
:1016F000029774F0809131029091320298878F8323
:101700001986BB86AA862C87CE0107960E945608AA
:1017100086E0F801A1E3B2E001900D928A95E1F72D
:101720000E94610A0E94520A0AC0231711F1C801DF
:101730000E94BD0881112CC0C8010E945608FF24D8
:10174000F394D1C05111F1CF7A2DB98AA88A522FC2
:101750006E2D89890E94D80881E392E00E94560884
:1017600086E0F60111928A95E9F70E94520AF12C5F
:10177000BAC04913DCCFE110DACFF8018583C80184
:101780000E94560886E0F60111928A95E9F7ABC0EF
:10179000EE2091F220913602822F82958F7090E098
:1017A00002970CF4B5CF80913102909132029A8366
:1017B00089831B82BD82AC822E83CE010196A6CF87
:1017C000E83CF10508F044C0FE2CEE2009F4B4CF4B
:1017D000231330C049132EC02091360220FD21C0B2
:1017E000822F82958F70482F50E041155105C9F026
:1017F000F80125834F30510541F08F5F982F929566
:10180000907F822F8F70892B8583C8010E94560894
:1018100086E0F801A1E3B2E001900D928A95E1F72C
:101820003DC086E0F801A1E3B2E001900D928A95F7
:10183000E1F759C0C8010E94BD08811169CF8091AC
:101840003602816080933602C8010E9456084BC060
:101850007A2DB98AA88A522F6E2D89890E94D808BC
:1018600086E0F60111928A95E9F718C0EE2009F496
:1018700063CFC8010E94BD08F82E882309F45CCF0D
:1018800086E0F801A1E3B2E001900D928A95E1F7BC
:1018900081E392E00E94A0050E94610A0E94520A20
:1018A00022C04D872E878D859E850E94050A292F8F
:1018B00022952F70223028F49F7039F0811105C0D5
:1018C0000BC0243028F49F7049F4805E883020F0EB
:1018D000C8010E9456089F2CF92C05C0F80195817B
:1018E000907F99F7F9CF8F2D6196EBE00C948B2ABE
:1018F000ACE0B0E0EEE7FCE00C94782A4F83588728
:1019000069877A878B879C87CE0107960E94C80AD1
:101910008823D1F09F8188852A853B85232B31F050
:101920008F3F31F481E09F3F19F403C081E001C093
:1019300080E080FD6FC04F81588569857A858B85F1
:101940009C850E94E20866C086E0FE013796DE01B3
:10195000119601900D928A95E1F7FF81E8856A85DD
:101960007B856115710531F0EF3F31F481E0FF3F78
:1019700019F403C081E001C080E080FD4BC080917C
:10198000000290E09C012F5F3F4F2770332740916A
:10199000FF0150E02417350709F443C0F983EA83B7
:1019A0007D836C8366E070E00E94CD29DC01AF5F2F
:1019B000BD4F96E0FE01319601900D929A95E1F7A8
:1019C000209300020E94330A25C090E066E070E098
:1019D0000E94CD298F5F9D4F0E94C80A882371F114
:1019E0008091FF0190E066E070E00E94CD29FC014B
:1019F000EF5FFD4F408151816281738184819581C8
:101A00000E94E2088091FF0190E00196877099277B
:101A10008093FF018091FF01909100028913D5CF3F
:101A20000DC00E949D08109200021092FF01E1E398
:101A3000F2E086E0DF011D928A95E9F72C96E2E05C
:101A40000C94942A80913F028595859585950895FB
:101A500080913F028770089590913F02977081E0D6
:101A600009F480E0089580914A02089590914A0215
:101A7000892B80934A020895809590914A02892388
:101A800080934A02089510924A0208959091490263
:101A9000892B80934902089580959091490289236A
:101AA000809349020895109249020895809140025E
:101AB000089508950E94590D08950E945A0D0895A1
:101AC0009091C20292FF08C090914002981721F0B5
:101AD000809340020E945D0D08958091400288230A
:101AE00029F01092400280E00E945D0D0895CF938E
:101AF000DF93E0910401F091050180914A02808317
:101B0000E0910401F0910501908180914902892BB7
:101B1000808380914002882381F0E0910401F0915C
:101B200005019081892B80838091040190910501AA
:101B30000E949B2181110E946D0DC0910401D091E2
:101B4000050148E050E067E372E0CE010E940A2BF5
:101B5000892B59F088E0FE01A7E3B2E001900D92D5
:101B60008A95E1F7CE010E944621DF91CF91089539
:101B70000E94590D08959091C20292FF11C0982FB2
:101B8000990F990F990F692B60933F020E942309C7
:101B900080913F028595859585950E94B80D0895A1
:101BA0000E942309089510923F0280E00E94B80D20
:101BB000089520913F028095822380933F02982FC1
:101BC000977099F430E0482F082E000C550B24171D
:101BD000350759F09091C20292FF07C0859585950F
:101BE00085950E942F090E94D30D08959091C202FD
:101BF00092FB222720F9281769F080FB92F9909335
:101C0000C2028091C1029091C2020E943F0E82E006
:101C10000E94D90D08958091C20282FB882780F925
:101C200091E089270E94F60D089581E00E94F60D4B
:101C3000089580E00E94F60D08956FEF7FEF80E039
:101C400090E00E94522B089580E090E00E942E2B9D
:101C5000873E9E4F19F40E94011B089580E008956D
:101C600082E090E00E94202B089583E090E00E94A3
:101C7000202B089584E090E00E942E2B0895BC0153
:101C800084E090E00E94522B0895AB01BC018FE0EC
:101C900090E00E94462B0895AB01BC0183E190E0E7
:101CA0000E94462B089560E070E0CB010E944C0E2C
:101CB000089560E070E0CB010E94450E0E94530E33
:101CC000089567EE7EEF80E090E00E94522B60E086
:101CD00082E090E00E94342B60E083E090E00E947C
:101CE000342B1092FE0160E074E184E090E00E94E9
:101CF000522B60E086E090E00E94342B6FEF87E08B
:101D000090E00E94342B40E050E0BA0188E090E07F
:101D10000E94462B60E08DE090E00E94342B40E072
:101D200050E0BA0188E190E00E94462B60E087E134
:101D300090E00E94342B40E050E0BA018CE190E04A
:101D40000E94462B60E070E080E290E00E94522BFF
:101D500040E050E0BA0188E190E00E94462B80E02C
:101D60000E941A1B0E944F1B0E94590E08950E9448
:101D7000610E0895682F8EE090E00E94342B089544
:101D80000E949E2260935B0270935C0280935D02CE
:101D900090935E02609357027093580280935902A9
:101DA00090935A02089581E008950E94D30E0895F9
:101DB00008950E94D80E08950E94D80E08950E949A
:101DC000DC0E08950E94D80E08950E94E20E089538
:101DD0000E94D80E08958EE891E10E942F210E9462
:101DE000E80E0E94E50E08950E94D90E0E94D80EBA
:101DF00008950E94AA110E94330508950E94892225
:101E00000E945F1B0E9483120E94F90E0E946319B8
:101E10000E94DF0E0895AAE0B0E0E1E1FFE00C943B
:101E20006D2A0E9499122DE4E22E22E0F22E570133
:101E3000D12CF501019111915F018D2D0E94C511E9
:101E400080279127D394F5E0DF1619F0892B89F3C9
:101E500022C0892B01F50E9492228C0180914B02B5
:101E600090914C020817190709F45BC08FEF898322
:101E70008A831B820E9492228160782F9D838C83AB
:101E800049815A816B818D810E945F0510934C02BC
:101E900000934B0246C080915F0281FD0E94CE11EB
:101EA0000E94D50E782E10E0812F0E94C5114C01A2
:101EB000F701A080B180A826B926A114B10449F188
:101EC00000E0CC24C394D12CC5018C219D21892B09
:101ED000C1F07720B1F00E831F8321E0C4018C2173
:101EE0009D21892B09F420E028870E94922281609D
:101EF000782F9A8789874E815F8168858A850E94BD
:101F00005F050F5FCC0CDD1C0E30F1F6F7019182FE
:101F100080821F5FF2E0EF0EF11C153029F60E945F
:101F2000C00E0E94A9190E9446052A96EDE00C9465
:101F3000892ACF93DF930E94AF10EC01811520E531
:101F40009207E0F5811530E4930708F09FC0803ECA
:101F5000910528F58D3C910508F096C0883A9105C9
:101F600070F4853A910508F085C08130910509F437
:101F70007EC008F4DCC0049708F0DCC0D8C0813C07
:101F8000910508F0D4C0C85AD0E0CC0FDD1FC95A63
:101F9000DE4F0990D881C02DCE019464CCC0C1150C
:101FA00080E2D80708F0B8C0C11591E0D90708F061
:101FB000C1C0C83ED10508F4BDC0B9C0803622E515
:101FC000920738F5803432E5930708F06CC0C032D0
:101FD00082E5D80708F05EC0C11592E5D90708F47C
:101FE0008AC04C2F4695469550E0F5E0440F551FAA
:101FF000FA95E1F7C37021E030E0C90102C0880F13
:10200000991FCA95E2F7EA01C82BD92BCE019D682A
:1020100092C0803A22E59207C0F48F71C03832E551
:10202000D30708F056C08695869590E065E0880F46
:10203000991F6A95E1F7C37021E030E002C0220FDA
:10204000331FCA95E2F73A6841C0C03C82E5D80721
:1020500008F446C0C03E92E5D90708F068C0CF71C9
:10206000DD27DC2FCC27CE01806F906A64C081E031
:1020700090E061C0C55AD0E0C757DE4F8881C82FB5
:10208000D0E0CE01906457C0906555C0DF70CE019E
:10209000906A51C0CF718C2F90E0D82FCC27CE0101
:1020A000816F906A48C08F718695869590E09C01FB
:1020B00075E0220F331F7A95E1F7C37081E090E05D
:1020C00002C0880F991FCA95E2F79C68822B932B58
:1020D00032C090E0D82FCC27CE01846F906A2BC0FD
:1020E0008C2F8F710E944B118F7190E0D82FCC27CD
:1020F000CE01906220C08C2F8F710E944B1195E011
:10210000D695C7959A95E1F7CF70D0E0DC2FCC2714
:10211000D0699E01282B09C08D2F8F710E944B1111
:10212000DD27D0628F719E01382BC90104C080E089
:1021300090E001C0CE01DF91CF910895753038F461
:102140006E3028F4462F672F0E946A1F089580E0A2
:1021500090E008950E949E100E94990F0895823881
:10216000910569F1B0F48133910509F475C048F423
:102170008932910509F467C08A32910509F471C06A
:1021800008958533910509F459C089339105B9F053
:102190000895833E910589F138F4803E9105D1F090
:1021A000823E910529F10895863E9105C9F1873E49
:1021B0009105D9F1843E910509F06CC027C02091AA
:1021C000C10220FD57C021FD55C02091C20223FD50
:1021D0005BC008958091C10280FD48C08091C20219
:1021E00080FF48C08091C10284FD46C083EE51C08B
:1021F0008091C10282FF3CC0F5CF8091C10282FD77
:1022000037C08091C20280FD35C0ECCF8091C20200
:1022100081FF36C08091C10284FD2EC087EE39C097
:102220008091C10283FF2AC0F5CF8091C10283FD56
:1022300025C08091C20281FD23C0ECCF8091C102F4
:1022400085FD22C01FC08091C10285FD1BC0809109
:10225000C20283FF19C00AC08091C10286FD16C068
:1022600017C08091C10286FD13C010C089E311C060
:1022700082EE0FC080EE0DC080E00BC086EE09C07C
:1022800084EE07C085E305C089E203C08AE201C08D
:1022900081E390E008959091C10292FF0DC0282F34
:1022A0002871283019F4877F846006C0282F247194
:1022B000243011F48B7F886093FF0DC0282F287184
:1022C000283119F4877E846106C0282F24712431B7
:1022D00011F48B7E88612091C20220FF0DC0382F3F
:1022E0003871383019F4877F816006C0382F31711A
:1022F000313011F48E7F886021FF0DC0282F2871A6
:10230000283119F4877E816106C0282F217121317F
:1023100011F48E7E886194FD877E089580E0089593
:102320000E941D0E08950E9499128FE39CE9019767
:10233000F1F700C000000E94991280E00E94C511D0
:1023400080FF04C00E9490110E94DF2208950E9425
:10235000931108950E94240E811102C00E94B70EAD
:102360000E94300E80935F020E943A0E9093C20248
:102370008093C1020E94A7110E94350E0E94F908A5
:102380008091FD010E940E090895E82FF0E0EE0F04
:10239000FF1FE353FD4F808191810895089580EAE6
:1023A0008A95F1F7089500C008950E94CF1108950D
:1023B00008950E94D81108950E94D91108950E948D
:1023C000D81108950E94DF110895F894E82FE2953E
:1023D000EF70F0E031A1282F2F7081E090E001C074
:1023E000880F2A95EAF7982F9095932391A392A1AD
:1023F000892B82A3789408950F931F93CF93DF9333
:10240000CAE9D1E089918F3F11F00E94E51181E086
:10241000CF39D807B9F7CCE8D1E00AE911E08991C2
:102420008F3F11F00E94E5110C171D07C1F7DF91D6
:10243000CF911F910F910895A0E0B0E0E2E2F2E1A8
:102440000C94712A8C01C62FD0E0CE0186569E4F87
:102450006C01FC0190819F3F09F450C0B62EF894A6
:10246000E92FE295EF70F0E081A19F7021E030E06C
:1024700001C0220F9A95EAF7822B81A382A12095B1
:10248000282322A378940E94D311ECE8F1E04AE9D2
:1024900051E021E030E0E12CF12C61916F3F89F0B7
:1024A000A62FA295AF70B0E090968C9190E06F70DF
:1024B00002C0959587956A95E2F780FD02C0C90133
:1024C00002C080E090E0E82AF92A220F331F4E175D
:1024D0005F0719F7F60180818F3F11F00E94E51127
:1024E00061E0E114F10409F460E08B2D0E94D51144
:1024F000CC0FDD1FC00FD11FF982E882CDB7DEB748
:10250000E9E00C948D2A0E94FC118AE0EDECF2E0E7
:10251000DF01982F1D929A95E9F7E3ECF2E0DF01D5
:102520001D928A95E9F785E00E94D4120E948F04DB
:102530000895AAE0B0E0EFE9F2E10C94752A8E016B
:102540000F5F1F4F8AE0F80111928A95E9F7F12C8D
:102550006F2DC8010E941C12F394F5E0FF12F8CF12
:102560004AE050E0B80183EC92E00E940A2B21E09F
:10257000009709F420E0892B41F08AE0F801A3ECF0
:10258000B2E001900D928A95E1F745E06DEC72E0C2
:1025900083EC92E00E94D512182F0E949204812FA2
:1025A0002A96E5E00C94912A0895EF92FF920F93FA
:1025B0001F93CF93DF937C018B01C42F222349F01B
:1025C00081E0809362020E94922290936102809344
:1025D000600280916202811102C080E01CC0809183
:1025E0006002909161020E94AA220597B0F3D0E0A8
:1025F000CC0FDD1FAE01B701C8010E940A2B892B49
:1026000039F0AE01B701C8010E94172B81E001C06B
:1026100080E010926202CDB7DEB7E6E00C94902A1B
:102620000E9467240E94FE0E0E94742408950E9456
:1026300079240E940B0F0E94932408950E942F2258
:102640000E944D240E94EB0E0E9410130E9417134B
:102650000E94F40EFBCFEF92FF920F931F93CF9344
:10266000DF93E82F71110AC0442321F0F0E0E45712
:10267000FB4FE4916E2F7E2F8E2F6CC0C62FD0E0C3
:10268000072F10E0282F30E0442329F0F901E45708
:10269000FB4F249130E0CE0166E070E00E94CD292E
:1026A000EE24EA94F12CB7010E94112ADB01CC0F31
:1026B000DD1FCB016BEA7FEF0E94CD298C0F9D1FA0
:1026C000C82FCC0FC80FC701801B910BB9010E9406
:1026D000CD29E92F492FD0E0CE01B8010E94CD29A4
:1026E000692F70E0C701861B970BB9010E94CD29A5
:1026F000F92FC7018C1B9D0BB8010E94CD29692FB2
:1027000070E0C701861B970BB9010E94CD29A2304A
:10271000B10591F038F4109759F01197C1F48E2F4C
:102720007F2F0CC0A430B10579F050F0169779F4E2
:10273000722F842FE92F0DC0892F7E2FE22F09C021
:10274000822F7E2FEF2F05C0822F792F02C0722F8C
:102750008F2F6E2FCDB7DEB7E6E00C94902A41E0C4
:102760000E942B13089508950E94AF130895CF93EC
:10277000DF93762FE901682F842F0E94B4137983A9
:1027800068838A83DF91CF9108958091D702282FA3
:10279000269530E02115310519F48170826005C05D
:1027A0002B32310524F0817084658093D70208951F
:1027B00088E090E00E94282B0895CF92DF92EF925C
:1027C000FF926B017C010E94C513B701A60188E04E
:1027D00090E00E94462BFF90EF90DF90CF900895FD
:1027E0006091D7027091D8028091D9029091DA025B
:1027F0000E94DD130895E7EDF2E083E0808311820B
:102800008FEF8283838314826081718182819381BF
:102810000E94DD1308958091D70280FF02C0869543
:10282000089580E008958091D70281700895909175
:10283000DB02933018F49F5F9093DB02882351F002
:102840006091D7027091D8028091D9029091DA02FA
:102850000E94DD13089581E00E941714089590915D
:10286000DB02992319F091509093DB02882351F0F9
:102870006091D7027091D8028091D9029091DA02CA
:102880000E94DD13089581E00E942F140895809125
:10289000DB0208958093DB02662351F06091D7023A
:1028A0007091D8028091D9029091DA020E94DD13D2
:1028B000089560E00E944A1408958091D802089516
:1028C0008091D90208958091DA02089570E00E9403
:1028D000D61A089530910A018091D70280FF0DC069
:1028E0008091090190E063E070E00E94CD29632FA0
:1028F00084529D4F0E946614089520910B014091CF
:102900000C01241768F7822F90E063E070E00E94CA
:10291000CD29FC01E452FD4F1182108212822F5FFB
:10292000F0CFA82FB62F8091D70280FF16C020913C
:102930000B0130910C01231770F4822F90E063E0BB
:1029400070E00E94CD29FC01E452FD4FA183B083C9
:1029500042832F5FF0CF0E946A140895A3E0B0E095
:10296000E4EBF4E10C94782A9091D70290FF0AC02E
:102970009E012F5F3F4F0E94B7134B8169818A816F
:102980000E9491142396E2E00C94942ACF93DF9353
:10299000EC01EC81F0E0E957FC4F4491E7EDF2E007
:1029A000628181810E94AE148C818F5F8C83DF9164
:1029B000CF910895CF93DF93EC01E7EDF2E04381EF
:1029C00062818C810E94AE148C818F5F8C83DF9139
:1029D000CF910895A3E0B0E0E0EFF4E10C94762A03
:1029E0008C018091630281110AC09E012F5F3F4FCD
:1029F0004FEF6FEF0E94B7138A8180936302F80153
:102A00008481813051F028F0823061F4409163027A
:102A10000AC08091630240E007C06091630240E019
:102A200080E003C040E080E060E00E949114F80183
:102A3000848190E0019663E070E00E94252A8483FF
:102A40002396E4E00C94922AA3E0B0E0EAE2F5E1F8
:102A50000C94702AF82ED62EE42EC22E9091D70216
:102A600090FF6EC0E92FE695AE2FB0E0A156BE4FA5
:102A70008C918093A9029E7F923061F49E012F5F1A
:102A80003F4F8F2D0E94B7134B8169818A810E942D
:102A9000911444C0823019F4E090DA023FC08630CD
:102AA00019F4F090D8023AC08930D9F38931B1F5E0
:102AB000E9514E2F4170B42EE695F0E0E957FB4FF7
:102AC000E491A12C0E2F10E040910D01A41620F5E9
:102AD0002A2D30E0C901B8010E94CD29642F70E091
:102AE0000E94112AEF2DB11002C0E60F01C0E61BB3
:102AF00080910B01A901480F511DCA0163E070E0EC
:102B00000E94CD299C0124523D4F4E2D6D2D8E2FBC
:102B10000E94B713A394D8CF0E946A14F092D802EF
:102B2000D092D902E092DA02CC2051F06091D70223
:102B30007091D8028091D9029091DA020E94DD133F
:102B40002396EAE00C948C2AE7EDF2E09181282F9D
:102B50004381628188E0890F0E942415089581E0F5
:102B60000E94A4150895E7EDF2E09181282F43819A
:102B7000628188EF890F0E942415089581E00E94E8
:102B8000B3150895E7EDF2E0628128E0620F08F4E2
:102B90006FEF282F438181810E942415089581E0E1
:102BA0000E94C2150895E7EDF2E0628128E0621B01
:102BB00008F460E0282F438181810E942415089544
:102BC00081E00E94D3150895E7EDF2E0438128E00B
:102BD000420F08F44FEF282F628181810E94241553
:102BE000089581E00E94E4150895E7EDF2E0438145
:102BF00028E0421B08F440E0282F628181810E9476
:102C00002415089581E00E94F515089520E00E94A2
:102C100024150895EF92FF921F93CF93DF93EC0159
:102C200010E0EE24EA94F12C30910D01131700F519
:102C300020910B01812F90E0820F911D63E070E0E5
:102C40000E94CD29FC01E452FD4F632F70E0C701C3
:102C50000E94252A812F0E94C4299C819F014091B6
:102C6000DA026091D902890F0E94B7131F5FDCCF8F
:102C70000E946A149A818C8190FF02C08F5F01C00C
:102C800081508C83DF91CF911F91FF90EF90089539
:102C9000A0E0B0E0EEE4F6E10C94702AFC01828141
:102CA00080FF02C0DFEF01C0D1E0C0E03CE0A32E16
:102CB00080910D01C81708F043C080910B01CC2E04
:102CC000D12C9601280F311DC90163E070E00E94EC
:102CD000CD2984529D4F7C01FC0111821082128209
:102CE00004E010E0B12C809165028B0D8D302CF04A
:102CF0006A2D0E94032A892F05C087FF03C0909187
:102D00000D01890F082E000C990BC816D90691F4F5
:102D10008091DA0290E0B8010E94CD2995958795BF
:102D2000959587959701482F6091D9028091D80297
:102D30000E94B713BD0E01501109A9F6CF5FB8CF9D
:102D40000E946A1480916502D13031F4811102C071
:102D500080910D01815007C090E0019660910D01B6
:102D600070E00E94252A80936502CDB7DEB7EAE0C5
:102D70000C948C2ACF9320910B0130910C012317D6
:102D800070F4822F90E063E070E00E94CD29FC0196
:102D9000E452FD4F1182108212822F5FF0CFC0E00B
:102DA00060910D01C61790F5EC2FF0E070E0CF01B7
:102DB0000E94252A90910B01890F20916402022E16
:102DC000000C330B90E063E070E00E94CD29E21725
:102DD000F307A4F020910801022E000C330B2E17EC
:102DE0003F0764F09C0124523D4F4091DA0260910C
:102DF000D9028091D8020E94B71306C0FC01E452A8
:102E0000FD4F118210821282CF5FCACF0E946A14D6
:102E10002091070180916402820F80936402909157
:102E20000801920F9093080119165CF4082E000C0B
:102E3000990B40910D0150E04150510984179507BD
:102E40001CF0219520930701CF910895A0E0B0E0F8
:102E5000ECE2F7E10C946A2A8C01FC01C481CC2ECF
:102E6000D12CE12CF12CA7019601C701B6010E94DB
:102E7000DE29A70196010E94DE294B015C0180E258
:102E800090E06C01CC1AD1080D2C000CEE08FF0864
:102E900025E530E040E050E0C501B4010E94DE29A4
:102EA0002B013C01A7019601C701B6010E94DE2952
:102EB000A70196010E94DE299B01AC01280D391D56
:102EC0004A1D5B1DC301B2010E94392AD22F822FF5
:102ED00090E02A3230F025E530E0A901481B590B7B
:102EE000CA0163E070E00E94CD2997FD0196959597
:102EF0008795C82FC095F12C85E5E82EED1A8091B5
:102F00000D01F816D0F4F1FC02C0EE2D01C0ED2F3A
:102F100020910B018F2D90E0820F911D63E070E0F6
:102F20000E94CD299C0124523D4F4C2F6091D90223
:102F30008E2F0E94B713F394E2CF0E946A14F80117
:102F40008481811102C091E003C0803219F49FEFA7
:102F50009093060190910601890FF8018483CDB703
:102F6000DEB7E0E10C94862A0F931F93CF93DF9393
:102F7000EC0100E010E040910D01842F90E0081773
:102F800019072CF580910B019801280F311DC901FB
:102F900063E070E00E94CD299C0124523D4F46958C
:102FA00050E08C81041715071CF4882331F002C00F
:102FB000811103C04091DA0201C040E06091D90262
:102FC0008091D8020E94B7130F5F1F4FD4CF0E9489
:102FD0006A148C8190E00196817099278C83DF912F
:102FE000CF911F910F910895A0E0B0E0EAEFF7E1D3
:102FF0000C946C2AFC017280648081E08483E7E891
:10300000F3E08490E6E0F4E0E491912CAA24AA9401
:10301000B12CE819EE2EF12C80910D01981608F0D4
:10302000A7C0092D10E022E0271570F0C80165E067
:1030300070E00E94CD29FC01EA59FD4F8091D80231
:1030400080838091D9028183C80165E070E00E948D
:10305000CD29611006C0FC01EA59FD4F138212828E
:103060006BC0EC01CA59DD4F8B81882321F181505F
:103070008B8390E06FEF70E00E94CD296C8170E04F
:103080000E94112AFB01FF27E957FC4FE4918E2F84
:10309000881990E06FEF70E00E94CD29B7010E947F
:1030A000112A2091DA0230E0862F90E0B9010E94C7
:1030B000CD299A8341C00E94ED2A9C018091DA02B9
:1030C0008695815890E062E071E00E94CD29C92E7A
:1030D000D12C2C153D0584F532E0371588F40E947B
:1030E000ED2AB5010E94252A88830E94ED2A2091AD
:1030F000D9022695622F70E00E94252A280F298385
:10310000C80165E070E00E94CD298A599D4FFC01FD
:1031100012822091DA02243120F0293C18F028ECA8
:1031200001C024E1C80165E070E00E94CD29FC01E6
:10313000EA59FD4F2483238380910B019801280FC6
:10314000311DC90163E070E00E94CD299C01245229
:103150003D4FC80165E070E00E94CD29FC01EA59AD
:10316000FD4F4281618180810E94B713939454CFB7
:103170000E946A14CDB7DEB7EEE00C94882AE7ED22
:10318000F2E080818E7F8083608171818281938172
:103190000E94DD131092AA020E946A140895E7EDBE
:1031A000F2E080818E7F80831092AA020E946A14CE
:1031B00008956091D702669570E04BE050E08EE094
:1031C00091E00E94FD2A892B19F481E08093AA02E4
:1031D0000E9492229093A3028093A202089590915C
:1031E000D70290FF35C09170811102C0926006C075
:1031F0008B3210F0946502C0880F982B9093D70201
:10320000662351F06091D7027091D8028091D90263
:103210009091DA020E94DD136091D702669570E00A
:103220004BE050E08EE091E00E94FD2A892B19F0DE
:103230001092AA0202C00E94D91881E08093A502D0
:103240004091DA026091D9028091D8020E9406165C
:103250000895682F9091D702969581E0890F8B325F
:1032600008F081E00E94EF18089581E00E9429197A
:103270000895682F9091D70296958FEF890F09F4E2
:103280008AE20E94EF18089581E00E94391908959A
:1032900061E00E94EF180895E7EDF2E0808181601F
:1032A000808386950E94481908958091D70280FFF7
:1032B00003C00E94BF1808950E944C19089560E051
:1032C0000E94EF1808958091A80281112EC00E94DB
:1032D000240E811104C00E94B70E0E94FB130E94AD
:1032E000D8136093D7027093D8028093D902909339
:1032F000DA026E7F61F40E94FB130E94D813609380
:10330000D7027093D8028093D9029093DA020E9478
:10331000C5131092AA028091D70280FF03C0869540
:103320000E945F1981E08093A8020895E7EDF2E022
:1033300080818160808386950E945F1908958091C5
:10334000D70280FF03C00E94CF1808950E949619EB
:1033500008950F931F93CF93DF938091AA02882340
:1033600009F491C08091A902E091D702E695E81B8B
:10337000E093A402823049F4F0E0ED57FC4FE49171
:10338000CE2FD0E006EC14E159C0863049F4F0E0CD
:10339000E058FC4FE491CE2FD0E00AED14E14EC08E
:1033A000893051F4E695F0E0E358FC4FE491CE2FDC
:1033B000D0E00AE016E142C08F3051F4E695F0E02B
:1033C000E658FC4FE491CE2FD0E008E416E136C079
:1033D000853149F4F0E0E958FC4FE491CE2FD0E07C
:1033E0000AEB16E12BC08831D9F0833239F4E5E7D6
:1033F000F3E0C591D4910AEE14E120C08432A9F023
:103400008532C1F48E2F63E00E94F729E92FF0E0A6
:10341000EE58FC4FE491CE2FD0E004EF17E10EC040
:10342000C8E2D0E006E217E109C0C4EFD1E004EB46
:1034300017E104C0C0EDD7E003EB13E18091A502D2
:10344000882361F01092A5020E9492229093A30219
:103450008093A2021092A7021092A6020E949222CA
:10346000E091A202F091A3028E1B9F0B8F3F9F471A
:1034700050F4EC0FFD1FF093A302E093A20282EA46
:1034800092E0F8010995DF91CF911F910F91089576
:10349000882311F0FA0101C0FB0109950895CF932B
:1034A000DF93C82FD62F0E940B148C1738F00E9480
:1034B0000B148D1718F40E94351903C08C2F0E942D
:1034C0004819DF91CF9108951F93CF93DF93FB01AC
:1034D0001281111166C0EC010E94330D8272FE014F
:1034E000E052F847E531F10508F05AC0EA5BFF4FBA
:1034F0000C945B2A0E94551954C044E459E165E3D9
:1035000079E104C045E359E164E479E10E94481A95
:1035100048C04EEB55E16FEA75E1F8CF4FEA55E14F
:103520006EEB75E1F3CF40EE55E16FEC75E1EECF58
:103530004FEC55E160EE75E1E9CF42E056E161EF15
:1035400075E1E4CF41EF55E162E076E1DFCF43E49E
:1035500054E16BE274E1DACF4BE254E163E474E1ED
:10356000D5CF81E015C065E082E017C068E086E055
:1035700014C06EE089E011C064E18FE00EC067E125
:1035800085E10BC088E104C062E289E106C083E204
:103590000E94481906C06AE285E20E944F1A01C0E3
:1035A00011E0812FDF91CF911F910895539A2BB194
:1035B000277F3BB138604FB7F894FC01CB0163E043
:1035C00070E00E94CD298E0F9F1FE817F90789F040
:1035D000519168E03BB9000000C057FF2BB9550F6F
:1035E000000000C000C000C02BB900C06A9591F770
:1035F000ECCF4FBF8FE594E00197F1F700C00000DA
:10360000089582E290E00E94202B823281F483E2CE
:1036100090E00E94202B823151F484E290E00E94DD
:10362000202B91E0883009F090E0892F01C080E0E4
:1036300081700895CF93C82F811102C06FEF01C030
:1036400062E282E290E00E94342BC11102C06FEF6F
:1036500001C062E183E290E00E94342BC11102C0FC
:103660006FEF01C068E084E290E00E94342BCF91BC
:103670000895089585E290E00E94202B682F70E065
:1036800080E090E008950895CF93C62F0E94431BD9
:103690006C2F85E290E00E94342BCF91089580E05A
:1036A0000E941A1B60E070E0CB010E94441B0E9444
:1036B000FD1E0E94BF1F81E00E941A1B08950E94F8
:1036C000391B0E943A1B0E94431B0E94011B81115F
:1036D00002C00E944F1B08950E949F190895CF9326
:1036E000FB01C281CC23E9F09C01225037472031F5
:1036F000310520F482500E94CF1F0CC08115F7E7DE
:103700009F0751F481E00E94230943E062E081E0D9
:103710000E948504C0E018C081309747A9F482E078
:10372000F2CF8115E7E79E0711F481E004C08130F4
:10373000974749F482E00E942F0943E062E081E06C
:103740000E94850401C0C1E08C2FCF9108952FEF16
:10375000FC012083089580E00895CF93DF93EC016E
:1037600088818230D9F078F4813021F50E94631489
:1037700090E06FEF70E00E94CD296FEF70E00E9443
:10378000112A698317C0833091F0843099F40E9424
:103790005D1489830E9460148A830CC00E941314F4
:1037A000882319F00E940B1404C080E002C00E941C
:1037B00047148983DF91CF910895CF93DF93EC0174
:1037C0008881823001F1A8F4813079F5898190E017
:1037D0006FEF70E00E94CD296FEF70E00E94112A18
:1037E000D62F0E946014C82F0E945D144D2F6C2F9D
:1037F0001AC08330A1F08430C1F40E946314482FB2
:103800006A81898110C08981811103C00E94CF180B
:103810000CC00E94961989810E945F1906C0898197
:103820000E94591402C00E940616DF91CF9108959C
:10383000FC019C012E5F3F4F9081983041F0993000
:1038400051F0973059F4C9010E94DD1B0895C90158
:103850000E94AD1B08950E94F01308958FEF80839E
:103860000895FC012181223019F40E94181C08954A
:103870000E94A71B0895EF92FF920F931F93CF937F
:10388000DF93EC01062F0E94AB1B8111B1C0E881D0
:103890008E2F90E0FC013197E331F10508F0A2C0D2
:1038A000E55AFF4F0C945B2A19828BE05EC0898138
:1038B000823089F030F4813009F094C00E949E2259
:1038C0000CC0833079F0843009F08CC01A821B82DE
:1038D0001C821D8289C00E943A1B9A838B837C8341
:1038E0006D8382C07E0110E0812F0E94C511F70117
:1038F000928383831F5FF2E0EF0EF11C1530A1F776
:1039000073C08981823039F0853009F06BC08A81BB
:103910000E946C1B69C06A817B818C819D810E94A1
:10392000612A0E94441B60C04B816A8189810E9488
:10393000C11E9C838D8358C02C813D813227232753
:1039400032274B816A8189810E94E21E4DC00E940C
:10395000FD1E4AC0602FCE010E94311C45C00E944E
:10396000761F24C00E94781F99838A833DC06B8193
:1039700070E089819A81AE014C5F5F4F982789275B
:1039800098270E947B1F30C06B8170E089819A81EB
:10399000AE014C5F5F4F9827892798270E949E1F92
:1039A00023C00E94BF1F20C00E94A81E89831CC084
:1039B0006B8170E089819A81AE014C5F5F4F9827DF
:1039C000892798270E94281F0FC06B8170E089818A
:1039D0009A81AE014C5F5F4F9827892798270E94F4
:1039E0004A1F02C08FEF8883602FCE010E945123AF
:1039F000CDB7DEB7E6E00C94902ACF93DF93FC01BD
:103A0000DB0112968C91882309F4DDC09F013057A9
:103A10002332310508F0D8C0EF010E943A0E90938E
:103A2000C2028093C102FE01E150F047E232F1058B
:103A300020F4E259FF4F0C945B2A8091C10281600F
:103A4000AAC08091C2028860B2C08091C102826027
:103A5000A2C08091C10220C08091C10288609BC039
:103A60008091C2021EC08091C2028260A0C080917B
:103A7000C102806190C08091C10280628CC080913F
:103A8000C102806488C00E949D088091C102806844
:103A900082C08091C102886084607DC08091C20232
:103AA0008260816084C08091C1028E7F74C08091E9
:103AB000C202877F7CC08091C1028D7F6CC08091E3
:103AC000C10220C08091C102877F65C08091C2027F
:103AD0001EC08091C2028D7F6AC08091C1028F7E1C
:103AE0005AC08091C1028F7D56C08091C1028F7BE8
:103AF00052C00E949D088091C1028F774CC0809176
:103B0000C102877F8B7F47C08091C2028D7F8E7FED
:103B10004EC08091C10282FB222720F991E09227BA
:103B200090FB82F990FB83F936C08091C202982FF6
:103B3000909591708E7F892B90FB81F938C0809190
:103B4000C10286FB222720F991E0922790FB86F99B
:103B500022C00E949D088091C10287FB222720F984
:103B600091E0922790FB87F916C081E001C080E0C8
:103B70000E94BA0E1EC08091C10284FB222720F948
:103B800091E0922790FB84F906C08091C102982FA2
:103B9000909590FB80F98093C1020BC08091C20286
:103BA00083FB222720F991E0922790FB83F98093F1
:103BB000C2028091C1029091C2020E943F0E0E94F7
:103BC0009D0880E001C081E0DF91CF910895A0E0E1
:103BD000B0E0EDEEFDE10C94732AE82FF0E0E4573D
:103BE000FA4FD490282F26952695269530E0F90196
:103BF000E45DF94F0491877010E0082E02C015951E
:103C000007950A94E2F701701127F901E45EF94F74
:103C1000E490F12C082E02C0F594E7940A94E2F7A0
:103C200091E0E922FF24F901E45FF94FC491D0E06B
:103C300002C0D595C7958A95E2F7C170DD270115B9
:103C4000110519F081EE0E94A605E114F10419F0A6
:103C500086EE0E94A6058D2D0E943906E114F1041E
:103C600019F086EE0E94F3050115110519F081EE99
:103C70000E94F305CD2B19F08CE20E943906CDB7D6
:103C8000DEB7E7E00C948F2AEF92FF921F93CF9359
:103C9000DF93EC01162F8881882309F453C081300B
:103CA00009F041C08981813041F47E0182E0E80E53
:103CB000F11C8A810E94390609C0823049F47E01D4
:103CC000E2E0EE0EF11C8A810E94A605E7012DC0FC
:103CD000833041F47E01F2E0EF0EF11C8A810E94F4
:103CE000F305F4CF843011F021961FC02A8122966B
:103CF00080E090E030E0205331092A30310548F46B
:103D00006AE070E00E94CD29820F931F21962881DE
:103D1000F1CF009751F0EFE9FFE03197F1F700C0E4
:103D200000000197F6CF0E94E71D2196812F88237E
:103D300009F4B1CFEFE9FFE03197F1F700C00000DF
:103D40008150F5CFDF91CF911F91FF90EF900895B3
:103D500084E00895E82F862F90E06CE170E00E94E7
:103D6000CD29242F30E0220F331F280F391F8E2F2B
:103D700090E06CE870E00E94CD29820F931F869638
:103D800008950F931F93CF93DF938430A0F4653091
:103D900090F44E3080F40E94AA1E8C010E94202BC9
:103DA00090E0D82FCC27C80101960E94202B9E01BD
:103DB000282BC90102C080E090E0DF91CF911F91D4
:103DC0000F9108950F931F93CF93DF93843080F466
:103DD000653070F44E3060F4E9010E94AA1E8C0137
:103DE0006D2F0E94342B6C2FC80101960E94342B3A
:103DF000DF91CF911F910F9108950F931F93CF9350
:103E0000DF93C0E0D0E010E000E00E94F30390E018
:103E1000C817D9073CF4402F612F8C2F0E94F5035F
:103E20009C0102C021E030E0402F612F8C2F0E94C6
:103E3000E21E0F5F0E3049F71F5F153029F72196FC
:103E4000C430D10501F7DF91CF911F910F910895F3
:103E5000EF92FF920F931F93CF93DF93EA017A01C2
:103E6000E60EF71E8C01C8018696CE15DF0569F0B7
:103E7000003322E0120720F40E94202B888301C027
